:020000040000FA
:04000000831222281D
:08000800831605158312101088
:1000100007308A0043080027A30001308A003C30E3
:1000200023020021A300003C031908282308013CF7
:1000300003191C28C30A08288316051183121014FB
:100040000C1009008316031331308F00831603133D
:10005000900183120313850107309900831603135F
:100060009F010030850083120330C0000430C100BE
:100070000030C2000030C3008312FF308F008E01B9
:100080000C10313090000515831603138D3092004B
:10009000831203131C309500831203133B3093002B
:1000A000831203138C1083120313053092008316FE
:1000B00003130511831283160C140B178B1783126D
:0200C0006028B6
:1002000082072D29FF343529FF34FF34542954291E
:1002100054295429542954295429FF34FF34FF34D4
:10022000FF343D29FF34FF344829BA29FF342529FA
:10023000FF34FF34FF34FF34FF34FF34FF34282908
:10024000FF34FF34FF34FF34FF340030C300003488
:1002500083160313051563000034C30AC00A40085F
:10026000063C0630031CC0000034C30AC00340082B
:10027000FF3C0030031CC000003407308A00C30A72
:100280004308C30A0027C10041033F39C1000034BD
:1002900007308A00C30A4308C30A0027C000063C8F
:1002A0000630031CC0000034A0000530A002410845
:1002B000A1000310A10D04308A00210808248F003A
:1002C000A10A210808248E0003104008A100A10DF6
:1002D000210DA100A10DA10704308A0020080024EF
:1002E000A10707308A00C30A43080027A000233C67
:1002F000031D7C29A10A712920082B3C031D82299A
:10030000A10A712920082D3C031D8829A103712908
:1003100020082E3C031D9B290E08A0000310A00CF2
:1003200020078E0003188F0A0F08A0000310A00CEE
:1003300020078F0071292108833C8330031CA10012
:100340000310A10D05308A002108002583169200B4
:10035000831206308A0021080026930005308A00A7
:10036000A10A21080025920006308A0021080026F3
:100370009500013407308A00C30A4308C30A0027E6
:10038000C10041033F39A1000310A10D04308A00D0
:10039000210808248F00A10A210808248E000030BB
:0403A000950001348F
:10080000820709340B3400340234043405340734CD
:1008100082078534EE34C234F734D7345034E134AF
:100820007C34E7349634EB34A834EE349034F0342E
:10083000BE34F2347034F334CB34F434E834F53469
:10084000D434F6349D34F7344834F734DD34F83496
:100850005F34F834D234F9343834F9349434F93418
:10086000E634FA343034FA347434FA34B234FA34C4
:10087000EA34FB341E34FB344F34FB347B34FB341A
:10088000A434FB34CB34FB34EF34FC341034FC346C
:100890003034FC344E34FC346934FC348434FC345D
:1008A0009C34FC34B434FC34CA34FC34DF34FC34BF
:1008B000F334FD340634FD341834FD342A34FD3469
:1008C0003A34FD344A34FD345934FD346834FD344F
:1008D0007534FD348334FD348F34FD349C34FD3461
:1008E000A834FD34B334FD34BE34FD34C834FD3493
:1008F000D234FD34DC34FD34E634FD34EF34FD34E1
:10090000F834FE340034FE340834FE341034FE343F
:02091000183499
:100A00008207EE340734E1340734D4340734C83471
:100A10000734BD340734B2340734A83407349E3465
:100A20000734963407348D340734853407347E34E4
:100A30000734763407347034073469340734633448
:100A400007345E34073458340734533407344F3492
:100A500007344A3407344634073442340734FC340C
:100A60000534EE340534E0340534D4340534C83468
:100A70000534BD340534B2340534A83405349E340D
:100A80000534963405348D340534853405347E348C
:100A9000053476340534703405346934053418343B
:100AA00007345E34053458340534143407341334B1
:100AB00007344A3405344634053442340534FC34B2
:100AC0000434EE340434E0340434D4340434C8340C
:100AD0000434BD340434B2340434A83404349E34B1
:100AE0000434953404348D340434853404347E3431
:100AF00004347634043470340434693404341834DF
:100B000005345E3404345934043454340434043425
:100B100007344A34043446340434423404343E3412
:100B200004340E3405340D34053434340434313493
:100B300004342E3404342C34043429340434093479
:100B400005342534043408340534213404340134A4
:020B5000073468
:100C0000820777341C3470343C346A341C346434C6
:100C10001C345E343C3459341C3454341C344F344A
:100C20001C344B341C3446343C3442343C343F3462
:100C30001C343B341C3438341C3434343C343134AC
:100C40003C342F341C342C341C3429343C342734A9
:100C50003C3425341C3423341C3421341C347E347D
:100C60001C3477341C3470341C346A341C346434BF
:100C70001C345E343C3459341C3454341C344F34EA
:100C80001C344B341C3446343C3442343C343F3402
:100C90001C343B341C3438341C3434343C340C3471
:100CA0001C342F341C342C341C340A341C340934C6
:100CB0003C3425341C3423341C3421341C347E341D
:100CC0001C3477341C3470341C346A341C3464345F
:100CD0001C345E343C3459341C3454341C344F348A
:100CE0001C344A343C3446343C3442343C343F3483
:100CF0001C343B341C3438341C3434343C340C3411
:100D00001C342F341C342C343C342A341C3402342C
:100D10001C3425341C3423341C3421341C341F343B
:100D20001C3407341C3406343C341A341C34183454
:100D30003C3417341C3416341C3414343C3404341E
:100D40003C3412343C3404341C3410343C3400340D
:020D50003C3431
:100E000082074F3403344C34103444342D34453489
:100E10002D344634473444342D3445342D3446344F
:100E2000473444344534463423344734233444343B
:100E30004534463423344734233444342D34453444
:100E40002D344634473444342D3445342D3446341F
:100E5000473444344534463423344734233444340B
:100E60004534463423344734233445342D34463412
:100E700047344134453446342334473423344134F1
:100E80002334463447344134423446342B344734D7
:100E90002B3441342B344F3404344334503408342D
:100EA0004C3408344F340334413441342334423415
:0E0EB0004F3404344C34023443345A345A3430
:02400E00E43399
:00000001FF
